:100224000114006401140014FF0003050A0F1419DB
:100234001E00FF0003050A0F14191E00FF0001022F
:10024400030508090A0B0C0D0E00FF0003050A0F35
:0E02540014191E003F065B4F666D7D077F6F1D
:100297000525E525C394644024E4F525051AE51AE8
:1002A700943C4019E4F51A051DE51D943C400EE405
:0E02B700F51D051BE51B94184003E4F51B2202
:1002C500E4FFE4FE74482FF8E6FD30E704D296809B
:1002D50002C296D29774482FF8ED25E0F6C2970E24
:0B02E500BE08E10FBF08DBD295C295F8
:0102F00022EB
:10039900E52330E1031203B5E52330E3031203CF6C
:0C03A9001203E9E52330E50312040322EF
:10041D00E54BB43F03E4F54BE54DB43F03E4F54D37
:09042D00E54FB43F03E4F54F2252
:10000E00E52BF46047E52B75F00A120337FF3395A5
:10001E00E0FE74582FF58274023EF583E493F54F9B
:10002E00E52B75F00A120337AFF0EF3395E0FE744F
:10003E00582FF58274023EF583E493F54EE5263093
:10004E00E005434E80800B534E7F8006754E407503
:10005E004F40E52CF46047E52C75F00A120337FF8C
:10006E003395E0FE74582FF58274023EF583E493C7
:10007E00F54DE52C75F00A120337AFF0EF3395E02E
:10008E00FE74582FF58274023EF583E493F54CE529
:10009E002630E105434C80800B534C7F8006754C17
:1000AE0040754D40E51B75F00A8490025893F54B50
:1000BE00E51B75F00A84E5F093F54AE52630E20576
:1000CE00434A808003534A7FE51D75F00A849002EF
:1000DE005893F549E51D75F00A84E5F093F548024D
:0200EE00041DEF
:0904610012000E1203990202C5FB
:1001A000E52BF46033E52B6023E4F533F52D432391
:1001B00002D291053BE53B7002053AC3943CE53A17
:1001C0009400401DE4F53AF53B152B22C291752DA4
:1001D000015323FD5326FE225323FD5326FEE4F54F
:0201E0002D22CE
:1001E200E52CF46033E52C6023E4F533F52F43234B
:1001F20008D292053DE53D7002053CC3943CE53CC6
:100202009400401DE4F53CF53D152C22C292752F59
:10021200015323F75326FD225323F75326FDE4F51A
:020222002F2289
:100436000537E537C394644009E4F5371201A01285
:0304460001E222AE
:1000F000E52320E06220B518432301E522C3940ADA
:100100004003E4F522AF220522EF90022C93F52B59
:1001100020B418432301E524C3940A4003E4F524E2
:10012000AF240524EF90023693F52C20B31343231C
:1001300001051BE51BC394184007E4F51BF51AF5F0
:100140002520B213432301051DE51DC3943C400740
:08015000E4F51DF51AF5252266
:0C044900E5B0543CFFBF3C035323FE22EF
:1003B500051CE51CC3941440035326FEE51CC39499
:0A03C500644006432601E4F51C2203
:1003CF00051EE51EC3943240035326FDE51EC3945C
:0A03DF00644006432602E4F51E22E6
:1003E900051FE51FC3943240035326FBE51FC39441
:0A03F900644006432604E4F51F22C9
:100403000520E520C3943240035326F7E520C39427
:0A041300644006432608E4F52022A9
:09046A00EF6003C2B022D2B022FF
:09047300EF6003C2B122D2B122F4
:10035900D5311C05290529EF3395E0FEC3E5299F11
:10036900EE6480F87480984003E4F529E4F53422BA
:10037900D5321C052A052AEF3395E0FEC3E52A9FED
:10038900EE6480F87480984003E4F52AE4F5362297
:1002F100E52D601CE5347013E52990022493FF126B
:10030100046AE529A393F5317534017F0402035989
:03031100D2B02245
:10031400E52F601CE5367013E52A90022893FF123E
:100324000473E52AA393F5327536017F0402037939
:03033400D2B12221
:03000B000202628C
:10026200C0E0C0F0C083C082C0D075D008438CB15A
:10027200438AE005471202971200F0120436120474
:10028200491204611202F1120314D0D0D082D08339
:05029200D0F0D0E032C5
:10015800E4F526F52375B0FF7590FF758901D28CFB
:10016800D2A9D2AF7530FF752EFF752CFF752BFF06
:10017800F545F546F543F544F53CF53DF53AF53BCF
:10018800F52AF529F528F527F524F522F536F5346D
:08019800F52FF52DF53380FE73
:03000000020455A2
:0C045500787FE400D8FD75814F0201584B
:10033700C2D530F707B2D563F0FF05F030E70CB24E
:10034700D5F4048463F0FF05F080018430D502F40E
:0203570004227E
:00000001FF
